:10000000830100308A000428203084002E300F2025
:1000100083010A128A11AA2F04068001840A0406A9
:06002000031D0C28003452
:100DF2008301A701A801032F000000000000A70A39
:100E02000319A80A2D082806031D092F2C082706F6
:100E120003190800FD2E8301AB00142FF230AC0041
:100E22000130AD00F92683120313AB0B0F2F08001C
:100E320096308301AB00292F871207163D30AC0094
:100E4200AD01F926071287163D30AC00AD01F92637
:100E5200AB0B1D2F08004B308301AB003C2F8712D8
:100E620007167B30AC00AD01F926071287167B30DE
:100E7200AC00AD01F926AB0B302F0800073083011F
:100E8200860483168604061002300C27861C4F2F18
:100E9200A008031D4F2FA001A00A01348618552F68
:100EA200200B552FA0010234061D5D2FA408031D3F
:100EB2005D2FA401A40A09340619632F240B632FA2
:100EC200A4010A3407308604831686048610023091
:100ED2000C27061C722FA308031D722FA301A30A5D
:100EE20007340618782F230B782FA3010834061D28
:100EF200802FA208031D802FA201A20A0534061921
:100F0200862F220B862FA201063407308604033077
:100F120083168604061102300C27061C962FA108A0
:100F2200031D962FA101A10A033406189C2F210B41
:100F32009C2FA1010434861CA42FA508031DA42FF5
:100F4200A501A50A0B3486180034250B0034A5012F
:100F52000C348B010730831603139C0006309F006C
:100F620085108B0180308100EF30860083120616D7
:100F72008B01CF30831687008312A501A401A30140
:100F8200A201A101A0013F27A600260BCA2F06122B
:100F9200C42F2608023A031DD02F0616C42F260896
:100FA200033A031DD62F8514C42F2608043A031DC5
:100FB200DC2F8510C42F2608053A0319F82F2608BE
:100FC200063A0319FE2F2608073A0319F82F2608B6
:100FD200083A0319FE2F2608093A0319F82F2608A2
:100FE2000A3A0319FE2F26080B3A031DFA2F192776
:0E0FF200C42F26080C3A031DC42F2C27C42F31
:02400E00323F3F
:00000001FF
